:020000040000FA
:02000000CD2B06
:08000800F500030EF6000A08E2
:10001000F7000A108A10831237083618B6183E30D7
:1000200081023308B407331C182836083320B4077C
:10003000340CB2003F39B21A403C5520321B103C00
:10004000B2000608F03932048600B60B2B283508BA
:10005000B300B114B6160B1177088A00760E830030
:10006000F50E750E09008207FF340034FF340034AA
:100070000034FF3400340034FF3400340034FF34E3
:1000800000340034FF3400340034FF3400340034D2
:10009000FF3400340034FF3400340034FF340034C3
:1000A0000034FF3400340034FF348207083408344D
:1000B0000934093409340A340A340A340B340B3451
:1000C0000B340C340C340C340C340D340D340D342E
:1000D0000D340E340E340E340E340E340E340F3410
:1000E0000F340F340F340F340F340F340F348B129E
:1000F00083165730810083128B1308000A304B237C
:10010000B7000830B50083165830810083128B1673
:100110008B170800B11C8A283508031C173CB50052
:10012000B1100800820755344E34493454347234C7
:10013000613463346B342034763430342E343934C3
:1001400000340339820700346434C8340F3982071D
:1001500000340A3414341E34283432343C344634E7
:1001600050345A34073982072434473450345234D7
:100170004D3443342C340739820724344734503407
:100180004734473441342C3482070034003401347E
:1001900006340134073401340334033400340034AA
:1001A00000340034003400340034003400340434AB
:1001B0000134820700340034003401340734083439
:1001C0000F3410341334003400340134073408344D
:1001D0000F3400340034003416341A348207A0344B
:1001E000A034A034A034A034603460342734763492
:1001F00058341C346C3420341C348400B901052973
:1002000084000008A120B900840A0008A620B907CC
:10021000840A00080F3939070800BA017B308400CE
:1002200030308000840A8000840A8000840A8000C4
:10023000840A80003C308400303080000408840A46
:10024000573A031D1C294E30C3004530CB003A08F5
:10025000573E84003A08EE208000BA0A3A080E3A67
:10026000031D2729CA2148215221CA29B800093073
:10027000390603195F29B908031D6F293A08B2200E
:100280003806031DCA29BA0A2C303806031D080097
:100290004C30840030308000840A0408523A031D38
:1002A0004A29B3295230840030308000840A80000B
:1002B000840A8000840A8000840A800008000A30D2
:1002C000390203186F293A08BB203806031D0800BD
:1002D000BA0A2C303806031D08005221B329380809
:1002E0002C3A0319B3293908C4203A060319080027
:1002F0003908073A031991293908083A031991294D
:100300003908123A0319912938082E3A03190800BE
:100310003908D9203A073C3E840038088000BA0AE0
:10032000080038082E3A0319AF293908D9203C3E75
:100330008400840A000884038000840A840A000878
:1003400084038000840A3908123A031DAC29840A08
:10035000000884038000840A3808800008003908F7
:10036000C420BA000800BA01B90A3908143A031DBA
:100370000800CD21523084000008FB00840A0008E8
:10038000FC00840A0008FD00840A0008FE00840ABC
:100390000008FF00BA01B90108003C308400273092
:1003A000DE000008413A0319D829703A031DDA2902
:1003B0006030DE00BB01840ABA01000DB9001A30BA
:1003C000840739081E3960388000E7308407BA0A8C
:1003D0003A08063A031DDD2906304B23BA00C03027
:1003E0003A1CD906BA1CD8063A1DD706C319DA0634
:1003F0004418DB06CB18DC0607304B233038DD0011
:100400000310DD0D4530FD201C3EDF004730FD2090
:100410001C3EE0004930FD201C3EE1004C30002134
:10042000E300E2010A30E20AE3020318132AE203BE
:100430006307A620E3006C30E2074F308400000819
:100440000F39203EE3075030FD201C3EE4004708F2
:100450000F393C300319E00745080F39031D080028
:100460005030DF07DB1B08000A30DF07DB175B13A8
:100470000800E80D680C8A2068091F39031D080070
:100480000310392A0030452A7E30E6000830E700A4
:10049000E60C3922E801E70B482A080001304B231B
:1004A000E500080008304B23E50008007E204222CA
:1004B000E50B572A4422FF30E900EA000800E60075
:1004C0000830E700660C01300318EA060310E90C57
:1004D000EA0C031C6F2A0830EA068430E906E60CB1
:1004E0003922E70B622A0800FF30EA066906E500B8
:1004F0006A085F2265085F224422442277200800B0
:10050000EB000000EB0B822A08008316051685110C
:10051000831285110800ED000A30EC0003108511EC
:10052000031C8515A930851E503080220314ED0C64
:10053000EC0B8F2A08000D30A42A08000A30A42AE8
:1005400008002030A42A08008B2AEE006E0EA92293
:100550006E080F39093C031CF93E393C8B2A6D109B
:10056000051E00340930EC003830851E1A30802218
:100570000310051E0314ED0CA930851E5030802297
:100580000000EC0BB82A6D08051AC42A6D14080087
:10059000AF226D1CC82A08008316851086128312AC
:1005A0000130F100F000FF30F300BB00F200080062
:1005B000061EF2016F080102EF07031C080003107A
:1005C000F00B08002630F000F20A0319F203061EB1
:1005D000F201BB0A0319BB03F10B08000A30F1005A
:1005E000F30A0319F3030800D822F2080319022BB7
:1005F00005304B237202031CFF2A8612032BF01EC8
:100600008612F01A86163B08053C03180E2B85103F
:100610005E08603A27300319DE00182B5E08603A46
:100620000319172B701A8514701E8510182B85144A
:100630000230061F09304B237302031C292B05309F
:100640004B2372020318252B4A2B4E22F301CA2199
:100650000134013E031D3F2BAB1B3D2BAB172B1071
:10066000AB108A30AA007A2529183D2B2B1489302B
:10067000AA007A25291CAB143D2B86174A2B023081
:10068000061F09304B23053C03184A2B7308013C15
:100690000319861300347F3983169B001C141A0833
:1006A000831208007F3983169B008B131C1555306D
:1006B0009D00AA309D009C141C118B179C185E2B6A
:1006C000831208004C300021B9010038031D6D2B46
:1006D000AE0A05302E02031C0800AE018617051570
:1006E00056225730840000085F22840A04085E3ACC
:1006F000031D732B00304B23AD002D084B23003816
:100700000319852B5F22AD0A7D2B00085F22840A26
:100710000408653A031D852B0F304B235F220E30F2
:100720004B235F22AC0BB42B03304B23AC002F3098
:100730005F2241305F223D305F227B085F227C08D0
:100740005F227D085F227E085F227F085F222030C3
:100750005F2204304B23AD002D084B2300380319D2
:10076000B42B5F22AD0AAC2B74220511080085144E
:100770008616BE2385108612BE2308000000AD0B2E
:10078000BE2BB70BBE2B08008B018316503086059D
:10079000831286170130B6000800831207309F00CD
:1007A00085220D21C4237720CC2226250530AE00DA
:1007B0008316051183120511B723B723B723013020
:1007C000AC00A201552CAF226D1CEC2BAD001B3AE6
:1007D0000319012C2D083621F42200380319E32BCC
:1007E000851A6223851AE32BBF24A20A0D304B23FE
:1007F0002202031CFD2BA201E32BFF30F300F201C8
:10080000E32BC822AD001B3A0319012C2D08443AF2
:1008100003193F2C2D08553A03194B2C2D08563A35
:100820000319552C2D08313A03195F2C2D08323A43
:100830000319622C2D08333A03196C2C2D08523AF7
:100840000319742C2D08723A0319A22C2D086E3A44
:1008500003197D2C2D08773A03198B2C2D08633A48
:100860000319BE2C2D08753A03191C2D2D08423A88
:1008700003198F2D2D08493A03192625E32BAD01C5
:10088000C82283169A0083122D085223AD0AAD1F89
:10089000402CCC22E32B8030A422AD012D084B2329
:1008A000A422AD0AAD1F4E2CE32BAD012D089220E2
:1008B000003803195E2CA422AD0A562CE32B051533
:1008C0007E20662C05157E2003108A20AF226D1C29
:1008D000662C77200511E32B05157E2003108A2056
:1008E000AF226D1C6E2C692CAD012D088400000810
:1008F000A422AD0A031D752CE32B3C30AD002D085E
:1009000084000008A4222D08AD0A653A031D7F2C3F
:100910009B229E22E32B83162130A0002008840016
:100920008312C8228316841780008413A00A201F14
:100930009D2CA01E9D2C201AA02C0D3A031D8E2C40
:100940008312E32B83162130A00020088400841733
:10095000000884138312A4228316A00A201FB42C3B
:10096000A01EB42C201ABA2C8417000884130D3A48
:10097000031DA52C83129B229E22E32BE32B8617BB
:100980000515562282305F22A0305F228A305F2216
:10099000AE305F22B0305F2260305F2260305F2275
:1009A00000304B23AD002D084B2300380319DB2CFE
:1009B0005F22AD0AD32C0B304B23AD002D084B2307
:1009C00000380319E62C5F22AD0ADE2C8316213095
:1009D000A000200884008417000884130D3A03192E
:1009E000FE2C84170008841383125F228316A00A4A
:1009F000201FE92CA01EE92C201EE92C83120C30AC
:100A00004B23AD0058305F2250305F224930AB1885
:100A100069305F2243302B1863305F2220305F2221
:100A20002D084B2300380319182D5F22AD0A102D15
:100A300074220511AB1308008030A422AD012D08EB
:100A40004B23A422AD0AAD1F1F2DE32B21308400C0
:100A5000841730308000840A8000840A8000840A71
:100A60002F308000840A30308000840A8000840A9D
:100A70008000840A67308000840A30308000840A55
:100A80008000840A8000840A74308000840A303038
:100A90008000840A8000840A8000840A2F3080004D
:100AA000840A4E308000840A6F308000840A5730F8
:100AB0008000840A58308000840A64308000840AF0
:100AC00061308000840A74308000840A61308000C4
:100AD000840A20308000840A0D30800084130800CE
:100AE0000000000000000000000000000000000006
:100AF0000000003412309F0070252A0883169F00E2
:100B0000831270251F1B29141F1F291007309F00F7
:100B1000702583160F309F00831270250034AB01BF
:100B2000AD0186168A30AA007A2529188616291C56
:100B30008612AD03031D922DAB03031D922D9B2244
:060B40009E228612E32B49
:02400E00023D71
:1042000010002800010001004500020000003000FD
:1042100028003C0040002100360001002F00620011
:104220009C009E00860082009800980060009C0020
:104230009E00A0008200A800900061000300F00032
:104240000000210035003000300030002E0030002A
:1042500030004E002F0030003100340033003000B9
:104260002E003000300045005F000000570058006D
:1042700054007200610063006B00200076002E0085
:10428000200030002E003900000055006E0069004B
:1042900054007200610063006B00200076002E0065
:0E42A000200030002E00390000000000000059
:00000001FF
